:020000040000FA
:10000000012885100510051185118316EF30810038
:1000100000308500FF308600831200308B0089019C
:100020000C3084008001840A041F1228041E122848
:10003000831200308B00103091000230900080302D
:100040008F001030940043309300C930920000308C
:100050008E0000308D0092308C002E281430A000CD
:10006000D92011089A009A0D9A0D9A0D0530A10019
:100070009A0D0318C128C328B120A10B38281008F5
:1000800099000830A100990D0318C528C728B12090
:10009000A10B43280F0898000830A100980D031801
:1000A000C928CB28B120A10B4E2805150000051149
:1000B00014089D009D0D9D0D9D0D0530A1009D0D09
:1000C0000318CD28CF28B120A10B5F2813089C006E
:1000D0000830A1009C0D0318D128D328B120A10B12
:1000E0006A2812089B000830A1009B0D0318D52830
:1000F000D728B120A10B75280515000005110E08A1
:100100009700970D970D970D0530A100970D0318D7
:10011000B528B728B120A10B86280D089600083015
:10012000A100960D0318B928BB28B120A10B912876
:100130000C0895000830A100950D0318BD28BF28B4
:10014000B120A10B9C28051500000511000000003E
:10015000000000000130A0008515D9208511640041
:100160002E28051400000510080085148A28851023
:100170008A2885149528851095288514A02885102F
:10018000A02885143C2885103C2885144728851014
:100190004728851452288510522885146328851015
:1001A000632885146E2885106E288514792885109B
:1001B00079289F0164009E0164009E0BDD289F0B3F
:0801C000DB28A00BD928080080
:02400E00F63F7B
:00000001FF
